:100000000C9411060C9471280C949E280C943906BB
:100010000C9439060C9439060C9439060C94390664
:100020000C9439060C9439060C94B60C0C943906D1
:100030000C9439060C9439060C9439060C94390644
:100040000C94CB280C9439060C94632C0C949E2CA5
:100050000C9439060C9439060C9439060C94390624
:100060000C9439060C943906D21BD91BD91BD21B10
:10007000D91BD91BD91BD91BD91BD91BD91BD91BE0
:10008000D91BD91BD91BD91BD91B471BD91BD91B62
:10009000D91BD91BD91BAA1AD91BD91BD91BD91BF0
:1000A000D91BD91BD91BD91BD91BD91BD91BD91BB0
:1000B000D91BD91BD91B531B531B531B531B531B3E
:1000C000531B531B531B531BD91BD91BD91BD91BA8
:1000D000D91BD91BAF1A521B521B521B521BD91BC7
:1000E000631B6B1B731B7B1B831B8B1B931B9B1B40
:1000F000A51BAF1BB91BC31BF61AB61AD91BD91BFC
:10010000D91BD91B471BD91BD91BD91BD91BD91BE1
:10011000D91BD91BD91B511B511B511B511BD91B5F
:10012000631B6B1B731B7B1B831B8B1B931B9B1BFF
:10013000A51BAF1BB91BC31BF61AB61AD91BD91BBB
:10014000D91BD91B471B0A1C0A1C0A1C0A1C0A1CA7
:100150000A1C0A1C0A1C0A1C0A1C0A1C0A1C0A1C6F
:100160002B1D2B1D2B1D2B1D2B1D2B1D511C5B1CFB
:10017000651C6F1CD51CDF1CED1CFF1C9C1D0C1E80
:10018000DD1DE21DE71DEC1DF11DF61DFB1D0C1E06
:10019000061E05251A2526252F253C2562256A25BC
:1001A0008D257A25456E746572206D656E752E2ECF
:1001B0002E00546F67676C6564206D6963726F50C1
:1001C000504D00546F67676C656420696E76657288
:1001D0007465642050504D2100546F67676C6564EE
:1001E000205458206D7574696E672100546F6767DD
:1001F0006C65642074656C656D657472792100505E
:10020000726F746F636F6C206572726F72207769A2
:1002100074682052580054696D656F757420776852
:10022000656E20636F6E6E656374696E6720746FB0
:1002300020525800507265737320616E79206B658F
:100240007920746F2063616E63656C00436F6E6E1E
:10025000656374696E6720746F2052582C20706F2C
:100260007765722075702074686520525820287751
:100270006974682062696E6420706C7567206966B5
:10028000206E6F74207573696E6720616C77617979
:10029000732062696E642900546F67676C6564201F
:1002A00027696D6D656469617465206F757470751B
:1002B000742700546F67676C65642027736C6176E0
:1002C00065206D6F64652700546F67676C656420F7
:1002D00027616C776179732062696E642700546FBF
:1002E00067676C65642050504D206368616E6E6571
:1002F0006C206C696D6974005365742052535349C6
:1003000020696E6A656374696F6E206368616E6EE2
:10031000656C2028303D3D64697361626C6529001D
:100320005365742050504D206D696E696D756D2058
:1003300073796E630053657420626561636F6E202C
:10034000696E74657276616C0053657420626561D4
:10035000636F6E2064656C6179005365742062651B
:1003600061636F6E206672657175656E6379206971
:100370006E20487A3A20303D64697361626C652C66
:100380002050783D504D52206368616E6E656C2040
:10039000782C2046783D465253206368616E6E6526
:1003A0006C2078005365742050574D2073746F7023
:1003B0002064656C61792028302064697361626C07
:1003C00065642C20312D323535203D3D20302E31D5
:1003D00073202D2035306D696E29005365742050CF
:1003E000504D2073746F702064656C6179202830E3
:1003F0002064697361626C65642C20312D3235355F
:10040000203D3D20302E3173202D2035306D696E1A
:100410002900536574206661696C736166652064A8
:10042000656C61792028302064697361626C656451
:100430002C20312D323535203D3D20302E3173209A
:100440002D2035306D696E29002A2A2A2A2A2A2A67
:100450002A2A2A2A2A2A2A2A2A2A2A2A2A2A2A2AFC
:100460002A2A2A2A2A2A0052582041636B656420CE
:100470002D2072657665727420737563636573737E
:1004800066756C21002A2A2A2A2A2A2A2A2A2A2A36
:100490002A2A2A2A2A2A2A2A2A2A2A2A2A2A2A2ABC
:1004A0002A2A002A2A2A2A2A2A2A2A2A2A2A2A2AD6
:1004B0002A2A2A2A2A2A2A2A2A2A2A2A2A2A2A2A9C
:1004C0000052582041636B6564202D207570646173
:1004D0007465207375636365737366756C21002A98
:1004E0002A2A2A2A2A2A2A2A2A2A2A2A2A2A2A2A6C
:1004F0002A2A2A2A2A2A2A2A2A2A2A2A0056616CE1
:1005000069642063686F69636573206172653A206E
:100510005B315D2D5B31365D20286368616E6E65F1
:100520006C20312D31362900536574206F7574703D
:10053000757420666F7220706F727420005B585D56
:100540002061626F7274206368616E6765732061F9
:100550006E64206578697420525820636F6E6669F6
:1005600067005B535D207361766520736574746901
:100570006E677320746F205258005B525D20726565
:10058000766572742052582073657474696E67734F
:1005900020746F2064656661756C747300557365B3
:1005A000206E756D62657273205B312D445D207421
:1005B0006F206564697420706F727473205B452DC1
:1005C000515D20666F722073657474696E67730085
:1005D000202D20726563656976657220636F6E6693
:1005E0006967757261746F722C207278207377203E
:1005F000000A0A6F70656E4C52536E672000536597
:10060000742073657269616C2062617564726174D3
:10061000653A200056616C69642063686F696365A0
:10062000733A2031202D20342B34202F2032202DDE
:100630002038202F2033202D20382B34202F203419
:10064000202D203132202F2035202D2031322B3407
:10065000202F2036202D203136005365742043682A
:10066000616E6E656C20636F6E6669673A20005339
:1006700065742044617461726174652028302D3284
:10068000293A200053657420486F70206368616EBA
:100690006E656C7320286D61782032342C20736570
:1006A0007061726174656420627920636F6D6D6141
:1006B00073292076616C69642076616C756573209E
:1006C000312D3235353A2000536574206368616EF0
:1006D0006E656C2073706163696E672028783130B5
:1006E0006B487A293A200053657420524620706F77
:1006F0007765722028302D37293A20005365742001
:100700005246206D616769632028686578292065F5
:100710002E672E20307844454144463030443A20FC
:10072000005365742062617365206672657175653A
:100730006E63792028696E20487A293A20005B5A36
:100740005D20656E74657220726563656976657299
:1007500020636F6E66696775726174696F6E20756C
:1007600074696C79005B465D20646973706C6179B3
:100770002061637475616C206672657175656E6366
:100780006965732075736564005B525D2063616CFD
:1007900063756C6174652072616E646F6D206B654A
:1007A0007920616E6420686F70206C697374005BDF
:1007B000495D207265696E697469616C697A65204A
:1007C00073657474696E677320746F20736B6574DE
:1007D00063682064656661756C7473005B585D20A6
:1007E000726576657274206368616E6765732061F7
:1007F0006E642065786974206D656E75005B535D6D
:1008000020736176652073657474696E67732074F4
:100810006F20454550524F4D20616E6420657869C8
:1008200074206D656E7500557365206E756D62651B
:100830007273205B302D395D20746F20656469749C
:1008400020706172616D657465727300202D205394
:10085000797374656D20636F6E6669677572617414
:10086000696F6E000A0A6F70656E4C52536E672096
:10087000005129204F7574707574206265666F721F
:1008800065206C696E6B20283D465329203A200074
:10089000502920536C617665206D6F646520286552
:1008A00078706572696D656E74616C293A20004FCD
:1008B000292054696D65642042494E4420617420AA
:1008C0007374617274757020203A20004E29205094
:1008D000504D206F7574707574206C696D69746506
:1008E0006420202020203A200044495341424C45B6
:1008F00044004D292050504D205253534920746FCD
:10090000206368616E6E656C202020203A20004CC8
:10091000292050504D206D696E696D756D20737979
:100920006E63202875732920203A200044495341E2
:10093000424C4544004B29204661696C73616665F1
:1009400020626561636F6E20696E74762E20283197
:100950002D32353573293A20004A29204661696CC9
:100960007361666520626561636F6E2064656C61AA
:10097000792028302D323535203D3E20313073200E
:100980002D203135306D696E293A200049292046E5
:1009900061696C7361666520626561636F6E206674
:1009A00072712E203A200048292050574D20737430
:1009B0006F702064656C6179202020202020203A0F
:1009C000200047292050504D2073746F70206465BB
:1009D0006C6179202020202020203A200046292008
:1009E0004661696C736166652064656C617920207D
:1009F00020202020203A200050574D206368616E4F
:100A00006E656C200066756E6374696F6E3A2000C7
:100A10002920706F727420004454462055484620A7
:100A200033322D6269742031306368004F70656E17
:100A30004C52536E675258206D696E6920342F36C0
:100A4000636800466C7974726F6E2F4F72616E67C7
:100A50006552582055484620386368005258207423
:100A60007970653A200044697361626C656400487E
:100A70007A00203D3D200043616C63756C617465B4
:100A800064207061636B657420696E746572766151
:100A90006C3A20004229204D6963726F20286861FA
:100AA0006C66292050504D202020203A00412920FA
:100AB000496E7665727465642050504D20696E20D1
:100AC000202020203A003029204D75746520627561
:100AD0007A7A657220286D6F73746C79293A0039BF
:100AE000292053657269616C20626175647261745A
:100AF000653A00736D617274506F72740046725380
:100B00006B79005472616E73706172656E7400442B
:100B1000697361626C65640038292054656C656D89
:100B2000657472793A202020202020200037292067
:100B30004368616E6E656C20636F6E6669673A200C
:100B40002000362920446174617261746520283068
:100B50002D32293A20202000352920486F7020634B
:100B600068616E6E656C733A202020202000342965
:100B7000204368616E6E656C2073706163696E6797
:100B80003A202000332920524620706F776572206A
:100B900028302D37293A20202000322920524620A3
:100BA0006D616769633A20202020202020202000EA
:100BB00031292042617365206672657175656E63C7
:100BC000793A2020200000000000240027002A009D
:100BD00000000000250028002B000000000023007A
:100BE000260029000404040404040404020202028E
:100BF00002020303030303030102040810204080E0
:100C0000010204081020010204081020000000075F
:100C100000020100000304060000000000000000C4
:100C2000462E11241FBECFEFD8E0DEBFCDBF13E0AC
:100C3000A0E0B1E0EEECFEE502C005900D92A63911
:100C4000B107D9F716E0A6E9B3E001C01D92A934B7
:100C5000B107E1F71CE0C2E2DCE004C02297FE012C
:100C60000E94422FC032D107C9F70E948B2E0C94EC
:100C7000652F0C940000A0E0B0E0E1E4F6E00C94F5
:100C8000112FEC01A880B980CA80DB80A114B104C7
:100C9000C104D10441F484E2A82E89EDB82E8BE57D
:100CA000C82E87E0D82EC601B5012DE133EF41E013
:100CB00050E00E94EE2E27EA31E440E050E00E942E
:100CC0009A2E7B018C01C601B5012DE133EF41E085
:100CD00050E00E94EE2ECA01B9012CEE34EF4FEF26
:100CE0005FEF0E949A2E6E0D7F1D801F911F97FF50
:100CF00004C06150704080409048688379838A8343
:100D00009B839B01AC015F77B901CA01CDB7DEB708
:100D1000EAE00C942D2F0E943B06089581EB92E0AF
:100D20000E943B0608956093B1027093B2028093D3
:100D3000B3029093B4020895A0E0B0E0E2EAF6E0D6
:100D40000C940A2FEC012B016A016115710519F051
:100D5000FB0191838083C114D10449F0C60102973D
:100D6000839728F020E030E040E050E0DCC0A9901C
:100D70008A2D90E00E945A2F892BC9F7FDE2AF1609
:100D800021F4A9903324339405C08BE2A81609F40A
:100D9000A9903324C114D10421F0E0E1CE16D1048E
:100DA00011F5F0E3AF1669F48881883711F08835C2
:100DB00041F4A980229682E0382A20E1C22ED12C6B
:100DC00012C0C114D10479F4E0E3AE1659F199E9E7
:100DD000E92E99E9F92E99E9092F99E1192F8AE06D
:100DE000C82ED12C3AC0FAE0CF16D10491F080E1A0
:100DF000C816D10429F0E8E0CE16D104F9F415C0E4
:100E0000BFEFEB2EBFEFFB2EBFEF0B2FBFE01B2F73
:100E100024C0A9E9EA2EA9E9FA2EA9E90A2FA9E135
:100E20001A2F1BC0F8E0CF2ED12CEFEFEE2EEFEFF4
:100E3000FE2EEFEF0E2FEFE11E2F0FC0960144277D
:100E400037FD4095542F6FEF7FEF8FEF9FEF0E949C
:100E5000CC2EC901DA017C018D0120E030E040E0B8
:100E600050E060E03601882477FC8094982C70ED87
:100E7000B72EBA0CF9E0FB1570F48A2D81548A3133
:100E800018F499ECB92E06C08A2D81568A3148F59E
:100E900089EAB82EBA0C8B2D90E08C159D050CF5C7
:100EA0006F3FE9F0E216F30604071507B8F0CA0130
:100EB000B901A40193010E949A2E9B01AC018B2DD4
:100EC00090E0A0E0B0E0280F391F4A1F5B1F2817F1
:100ED00039074A075B0710F061E001C06FEFA99086
:100EE000C6CF4114510451F0662311F0219703C07D
:100EF00031FE04C02297F201D183C08330FE07C0C7
:100F000050954095309521953F4F4F4F5F4F67FF6C
:100F10000AC082E290E090934806809347062FEF44
:100F20003FEF4FEF5FEFB901CA01CDB7DEB7E1E1A7
:100F30000C94262FFC0188279927E89421912032D0
:100F4000E9F3293010F02E30C8F32B3241F02D3266
:100F500039F4689404C00E94EF07820F911D21911B
:100F600020532A30C0F31EF4909581959F4F089529
:100F700046E953E00E94BD070895009731F4DA0175
:100F80008D919C91009709F40EC0DC01FB013D910D
:100F90002191222319F03217C9F3FACF332331F408
:100FA000DA011D921C928827992708951197AF9313
:100FB000BF93FB013D912191321771F4332321F44A
:100FC00088279927119702C01E921196FA01A193C2
:100FD000B0839F918F910895222369F7EACF7AE039
:100FE000979F902D879F802D910D112408958091BA
:100FF0009803813019F482E08093980380919803DC
:10100000833019F484E0809398030895009721F1C8
:101010009C0140E050E068E478EE81E090E00E94BE
:10102000EE2EC901DA018F3F9105A105B10531F01E
:1010300028F08FEF90E0A0E0B0E008C00097A10595
:10104000B10521F481E090E0A0E0B0E08093B3002E
:101050008091B000806103C08091B0008F7E80934A
:10106000B0000895E3E0F0E089E0809357008491B8
:1010700090E08670863009F491E0892F08951F93DF
:10108000182F0E943208882379F09FB781E080935F
:101090008F05F894A89588E1809360001093600014
:1010A000112309F0A8959FBF1F910895382F20E0C4
:1010B00080912105909122058227932740E061E2EB
:1010C00070E19C01220F331F97FF04C0C9018627DE
:1010D000972701C0C9014F5F483099F790932205C7
:1010E00080932105089586E38093BE0380E092EC0F
:1010F000A1E0B0E08093BF039093C003A093C1032D
:10110000B093C20387E08093CB0380EC92E9ADEE0D
:10111000B9E18093C3039093C403A093C503B09334
:10112000C60385E08093CC038DEE9EEFADEABEED65
:101130008093C7039093C803A093C903B093CA03D5
:10114000ADECB3E080E090E0863010F0E0E004C069
:10115000FC01E058FC4FE081ED9301968831910548
:1011600099F782E08093E5038AE08093E60308958F
:1011700080EC91EDA8E9BBE180939B0390939C03E5
:10118000A0939D03B0939E0310929F031092A0031F
:101190001092A1031092A20308958436910520F4C1
:1011A000BC0180E090E025C08E3B910550F48A554B
:1011B0009040BC0180E090E02AE030E040E050E068
:1011C00016C0823D910550F4845B9040BC0180E0E4
:1011D00090E024E630E040E050E009C08D5C9040B3
:1011E000BC0180E090E028E532E040E050E00E9461
:1011F0009A2E24E630E040E050E00E949A2E0895B6
:1012000090E08C599F4F0E94CD080895DC0198967C
:10121000EC91F0E0E770F070E858FC4F80810895A1
:101220008F929F92AF92BF92CF92DF92EF92FF92F6
:101230000F931F938C010E940609D80197962C9159
:1012400030E043E150E0249FF001259FF00D349FF2
:10125000F00D1124EB54FD4F80809180A280B3806B
:1012600090E00F96AA2797FDA095BA2FBC01CD015B
:1012700020E43FE14DE750E00E949A2EA501940141
:101280000E94CC2E69017A0180ED97E0A0E0B0E0E9
:10129000C80ED91EEA1EFB1ED80198968C91887143
:1012A00081F060E07EEE8AEB9BE0A50194010E9454
:1012B000CC2E28513C4F4F4F5F4FC20ED31EE41E21
:1012C000F51E87EE93E0A0E0B0E0C80ED91EEA1E3E
:1012D000FB1EC701B60128EE33E040E050E00E945B
:1012E000CC2ECA01B90128EE33E040E050E00E9464
:1012F0009A2E1F910F91FF90EF90DF90CF90BF90AB
:10130000AF909F908F9008958F3F910509F010F452
:1013100080E0089522E08030920710F481E0089583
:101320008050934010F083E0089582E00895CF92BA
:10133000DF92FF920F931F93CF93DF93F82FEB0170
:101340006A01182F1695E0E088819981D6018C9367
:101350008A819B8111968C9311978C819D81129625
:101360008C9312978E819F8113968C93139728816B
:1013700039814A815B816C817D818E819F819295CB
:10138000990F990F907C832F8370982B852F8370F2
:10139000880F880F982B872F83708295807F982BDA
:1013A00014969C9385E090E0C80ED91E2896EF5FB6
:1013B0001E1750F6F0FF21C0888199810E94840990
:1013C000F82E8A819B810E948409182F8C819D812F
:1013D0000E948409082F8E819F810E948409F294C3
:1013E000FF0CFF0C70ECF7221295107F1F29182BB1
:1013F000000F000F012BD6010C93DF91CF911F91AD
:101400000F91FF90DF90CF90089523E080329207F4
:1014100018F420E030E026C023E0883E920748F42C
:101420009C012F51334054E0369527955A95E1F7AA
:1014300019C027E0803D920720F49C012C5D3340C9
:1014400011C028E08839920718F02FEF33E00AC066
:101450009C01285C374044E0369527954A95E1F792
:101460002D503C4FC90108959C013695279525754F
:101470003575821B930B9C013695279536952795DC
:101480002373337383739373280F391FC901E4E007
:1014900096958795EA95E1F7820F931F8F709F705D
:1014A00021E031E0AC01429FC001439F900D529F6B
:1014B000900D1124892F0895882339F02D9800006C
:1014C0002B9A00002D9A000008952D9800002B986B
:1014D00000002D9A000008952D9A000083B12D98E8
:1014E000000090E0B4E096958795BA95E1F7817099
:1014F00008950F931F93082F5C9A2D985C9810E025
:10150000802F80780E945C0A000F1F5F1830C1F79F
:101510002D981F910F9108958F770E94790A089551
:101520000F931F93082F10E0802F80780E945C0A91
:10153000000F1F5F1830C1F72D981F910F9108956C
:101540000F931F932D9880E000E0182F110F0E9439
:101550006C0A810F0F5F0830C1F71F910F9108953A
:101560000E948C0A0E94A00A5C9A08951F93162F6D
:1015700080680E94790A812F0E94900A5C9A1F91CC
:1015800008951F931091C7031827EEEBF3E0E80FBF
:10159000F11D89E767850E94B60A8DE3612F0E94DD
:1015A000B60A82E4612F0E94B60A1F91089586E26E
:1015B0000E94B00A08950F931F938C018CE1F801EB
:1015C00064810E94B60A8DE1F80165810E94B60A25
:1015D0008EE1F80166810E94B60A80E2F801678117
:1015E0000E94B60A81E2F80160850E94B60A82E292
:1015F000F80161850E94B60A83E2F80162850E94C3
:10160000B60A84E2F80163850E94B60A85E2F80111
:1016100064850E94B60A8AE2F80165850E94B60ACE
:101620008EE6F80166850E94B60A8FE6F8016785A6
:101630000E94B60A80E7F80160890E94B60A81E735
:10164000F80161890E94B60A82E7F80162890E9466
:10165000B60A1F910F910895EF92FF920F931F9377
:10166000CF93DF937B018C01603028E372072CE974
:1016700082072CE1920728F520E836E948E950E096
:101680000E94CC2EE9016897B90180E090E020E843
:1016900039E647E65FEF0E949A2E6E0D7F1D801F90
:1016A000911F32E0660F771F881F991F3A95D1F777
:1016B00021E732E040E050E00E94CC2E890180E436
:1016C00021C020E03DE241E351E00E94CC2EE9013F
:1016D0006897B90180E090E020E033ED4EEC5EEFDA
:1016E0000E949A2E6E0D7F1D801F911F660F771F1F
:1016F000881F991F21E732E040E050E00E94CC2E85
:10170000890180E69E012F71622F680F85E70E9494
:10171000B60A86E7612F0E94B60A87E7602F0E940B
:10172000B60ACDB7DEB7E6E00C94312F9F92AF92A8
:10173000BF92CF92DF920F93DF93CF9300D000D070
:10174000CDB7DEB7982E83E00E94B00A8093E703FE
:1017500084E00E94B00A8093E80386E060E00E9483
:10176000B60A87E061E00E94B60A89E06FE70E944E
:10177000B60A8AE065E00E94B60A8BE065E10E9445
:10178000B60A8CE062E10E94B60A8DE06DEF0E941D
:10179000B60A8EE060E00E94B60A992019F084E152
:1017A00093E008C08091E50323E1829FC0011124EA
:1017B0008B549D4F0E94DB0A80E36CE80E94B60ABE
:1017C00082E36FE00E94B60A83E362E40E94B60AF5
:1017D00084E36AE00E94B60A85E36AE20E94B60AE0
:1017E00086E36DE20E94B60A87E364ED0E94B60AC2
:1017F00088E360E00E94B60A89E360E00E94B60ACE
:10180000992049F065E7A62E61ECB62E61ECC62E54
:101810006EEDD62E08C0A090C703B090C803C0904C
:10182000C903D090CA030AE38D2D9927AA27BB27A5
:1018300089839A83AB83BC83802F69810E94B60A17
:10184000802F8B5F69810E94B60ADC2CCB2CBA2CCE
:10185000AA240F5F0E3341F783E46FEF0E94B60AAC
:1018600084E46FEF0E94B60A85E46FEF0E94B60A27
:1018700086E46FEF0E94B60A992019F08DE666E0C3
:1018800003C08DE66091CB030E94B60A89E760E051
:101890000E94B60A8AE76091CC030E94B60A83E7E9
:1018A00060E00E94B60A84E760E00E94B60A9920D0
:1018B00029F060EC72E98DEE99E108C06091C303F4
:1018C0007091C4038091C5039091C6030E942C0BB4
:1018D0000F900F900F900F90CF91DF910F91DF90AD
:1018E000CF90BF90AF909F90089587E061E00E94F5
:1018F000B60A8EE764E20E94B60A88E063E00E94BE
:10190000B60A88E060E00E94B60A87E065E00E94BF
:10191000B60A85E062E00E94B60A83E00E94B00A3F
:101920008093E70384E00E94B00A8093E80308955F
:10193000582F40918C04842F90E0FC01EF70F070E0
:101940009F012F5F3F4F74E0959587957A95E1F75A
:101950002817390751F0E458FB4F5083842F8F5FCD
:101960008F70407F842B80938C0408951F920F9278
:101970000FB60F9211241F932F933F934F935F93B2
:101980006F937F938F939F93AF93BF93CF93DF9387
:10199000EF93FF93C0918600D09187002091CE04F1
:1019A0003091CF048091AD04882309F047C0CE0167
:1019B000821B930B9C0180919F0385FD02C036958D
:1019C000279599E0253C390708F180914703863037
:1019D000D0F0809147038F3FB1F020E00EC0E22F9E
:1019E000F0E0EE0FFF1FDF01A255BB4F8D919C91E0
:1019F000E95DFC4F918380832F5F80914703281717
:101A000070F31092AC041092470318C082E02D3B93
:101A1000380760F180914703803140F5109147030A
:101A2000C9010E94050AE12FF0E0EE0FFF1FE25509
:101A3000FB4F918380831F5F10934703D093CF04A4
:101A4000C093CE04FF91EF91DF91CF91BF91AF9101
:101A50009F918F917F916F915F914F913F912F91C6
:101A60001F910F900FBE0F901F9018958FEF8093CE
:101A70004703E4CF83E0809380008AE9809381006C
:101A800080919F0386FD05C08091810080648093D2
:101A900081008FEF9FEF9093890080938800809161
:101AA0006F00806280936F0008956F3020F08695FC
:101AB0008695805408958DE0689F802D11240895A7
:101AC000882319F460E071E002C063E071E085E210
:101AD00096E00E944E2C0895A0E0B0E0E2E7FDE021
:101AE0000C94132F182F0E9421299B01AC01809187
:101AF0001B0590911C05A0911D05B0911E05690163
:101B00007A01C81AD90AEA0AFB0AD701C60189581C
:101B10009341A040B04010F010921A0520931B058D
:101B200030931C0540931D0550931E052091AD0474
:101B3000822F81508230E8F580911A05882309F4BC
:101B40004FC1813011F482E0BCC1803108F035C151
:101B5000E82FF0E0E255FB4F10838F5F80931A056A
:101B6000803109F0B0C1A0EBB4E0213039F4119616
:101B7000EC911197E695E6958C9109C08D919C9119
:101B80001197E92FE695E695E69596958795E031CC
:101B900040F4F0E090E0EE0FFF1FE95DFC4F918311
:101BA00080831092AC04129684E0AE3BB807E9F64D
:101BB0008AC1233009F004C180911A05882321F4D9
:101BC0001F3009F080C10CC1883130F4E82FF0E0FB
:101BD000E355FB4F108374C1883109F0EEC0112327
:101BE00009F0EBC0C0E0D0E00BE010E0DE0163E004
:101BF000AA0FBB1F6A95E1F7C09FB001C19F700D8E
:101C0000D09F700D1124FB01E255FB4F8081218193
:101C1000922F977095958795FD01EE0FFF1FE95D57
:101C2000FC4F91838083FB01E155FB4F308136955A
:101C3000369536952181422F4295440F407E842F60
:101C4000832B269526952695922F977095958795A7
:101C5000FD01EE0FFF1FE75DFC4F91838083FB01C9
:101C6000E055FB4F808182958695869583704181F2
:101C7000942F990F990F292F282B42954695469519
:101C8000437082818170880F880F382F342B3595EF
:101C90002795FD01EE0FFF1FE55DFC4F318320838B
:101CA000FB01EE54FB4F308136952181422F479541
:101CB00044274795842F832B2695922F97709595CF
:101CC0008795FD01EE0FFF1FE35DFC4F918380833D
:101CD000FB01ED54FB4F308132953F702181422F43
:101CE0004295407F842F832B22952F70922F9770DF
:101CF00095958795FD01EE0FFF1FE15DFC4F9183E8
:101D00008083FB01EC54FB4F8081881F8827881F4C
:101D10004181942F990F292F282B441F4427441FBA
:101D200082818370880F382F342B35952795FD01DC
:101D3000EE0FFF1FEF5CFC4F31832083FB01EA5461
:101D4000FB4F3081369536952181422F4295440FC5
:101D5000440F407C842F832B26952695922F9770D5
:101D600095958795AA0FBB1FFD01ED5CFC4F9183F4
:101D7000808369547B4FFB01208122952695277033
:101D80004181342F330F330F330F832F822B942F46
:101D900092959695977095958795AB5CBC4F1196EB
:101DA0009C938E932196C230D10509F01FCF80916C
:101DB000C40483FD02C01092AC0410921A0583C0C3
:101DC000243009F080C040911A05442359F4183A90
:101DD000B1F4109222051092210588EA0E9456085B
:101DE00081E06FC0413019F410931F0504C04230E8
:101DF00031F410932005812F0E9456085DC0609138
:101E00002005262F30E0220F331FE42FF0E0C90118
:101E100002968E179F0734F0433268F7E555FB4F63
:101E20001083E9CF2D5F3F4F40912105509122054E
:101E3000E217F30749F4912F80E048275927509380
:101E400022054093210538C0812F90E0481759079B
:101E500089F580911F05813069F5613118F080E1C5
:101E600080932005D09020054EEAE42E44E0F42E25
:101E700000E010E01BC0F701D081C0E0818190E05C
:101E80008C2B9D2B33E0969587953A95E1F70E9430
:101E9000050AF801EE0FFF1FE95DFC4F9183808377
:101EA0000F5F1F4F82E090E0E80EF91E0D1518F34A
:101EB0001092AC0410921A0580911A05882319F02B
:101EC0008F5F80931A05CDB7DEB7E8E00C942F2F13
:101ED000FF920F931F93CF93DF93182F092FF62EA6
:101EE0008EE30E94B60A212F302FC901EC0110E0C9
:101EF00005C08FE769910E94B60A1F5F1F15C8F3DE
:101F000085E064E00E94B60A83E00E94B00A8093F4
:101F1000E70384E00E94B00A8093E8030E9421292D
:101F20006093E9037093EA038093EB039093EC03CF
:101F300087E069E00E94B60A81E080939803CDB7FC
:101F4000DEB7E5E00C94322F0E94680F8091980371
:101F50008130D9F40E9421292091E9033091EA03CC
:101F60004091EB035091EC03621B730B840B950BB8
:101F7000605A76488140904040F4E8CF85E296E090
:101F800067E071E00E944E2C0895809198038130A3
:101F9000A9F3089585E296E06EE70E94062E089563
:101FA000A0E0B0E0E6EDFFE00C94122F6C0185E2BA
:101FB00096E06EE70E94062E760100E010E0C0E099
:101FC000D0E0B0E2BB2E0AC00830110521F49E011A
:101FD0002095F60120870894E11CF11CF70160812F
:101FE000862F8D57823040F485E296E06DE70E949F
:101FF000062EF70160816B2585E296E00E94062E91
:102000000115110551F0F70180819E01280F311D46
:10201000C32FDD27C20FD31FD0700F5F1F4F0930B2
:10202000110591F6CDB7DEB7E9E00C942E2FA9E0AB
:10203000B0E0EDE1F0E10C94192F382FE62F8091FC
:10204000910490E0019664E270E00E94B92E982F0E
:102050008093910488E9898380E18A83913071F0CB
:10206000913028F0923099F09330E1F416C085E079
:102070008B8381EF8C832F5F2D8317C09B8381EF30
:102080008C8384E6489FC00111249D830EC084E0A8
:102090008B8381EF8C833D8308C09B8381EF8C838E
:1020A000ED8303C00E94CA0F04C0CE0101960E94B6
:1020B000D00F2996E2E00C94352F0F931F93CF9306
:1020C000DF93182F092F85E296E06EE70E94062E17
:1020D000212F302FC901EC0110E000E288818D57DB
:1020E000823040F485E296E06DE70E94062E8881FA
:1020F0008027888385E296E069910E94062E1F5F03
:10210000193061F785E296E06EE70E94062EDF91B6
:10211000CF911F910F910895A9E0B0E0E2E9F0E1BD
:102120000C94192F382F80919104882379F48EEF25
:1021300089833A836B83842F90E0959587958C8370
:102140002D83198618861F821E822FC040918C0411
:10215000842F90E09C012F70307054E09595879506
:102160005A95E1F78217930721F18DEF89831A823F
:102170001B82DE01149620E008C0E458FB4F8081EA
:102180008D93405F2F5F263069F0842F90E0FC0133
:1021900034E0F595E7953A95E1F78F709070E81780
:1021A000F90759F740938C042A83CE0101960E94C7
:1021B0005D108091910490E0019666E070E00E94CD
:1021C000B92E809391042996E2E00C94352F9F92CA
:1021D000AF92BF92CF92DF92EF92FF920F931F9335
:1021E000B82EA62ED42EC22E902E0E9421297B011D
:1021F0008C0180917B0420918D0430918E0440915C
:102200008F04509190048823B1F0D801C701821B3C
:10221000930BA40BB50B815E9E42A040B04020F111
:102220002C2DDC1408F42D2D8B2D6A2D422F292DF9
:102230000E94171011C0D801C701821B930BA40B79
:10224000B50B81539547A040B04070F08B2D6A2D9F
:102250004D2D2C2D0E948C10E0928D04F0928E0456
:1022600000938F04109390041F910F91FF90EF90B3
:10227000DF90CF90BF90AF909F90089585E296E059
:102280006091EE030E94062E08951F93182F85E299
:1022900096E0612F0E94062E8091EE0381278093A5
:1022A000EE031F9108951F93192F0E944511812F4E
:1022B0000E9445111F910895DF92EF92FF920F93B4
:1022C0001F93D82E7B011092EE0305E216E0C801A1
:1022D00065EB0E94062EC80162E60E94062E8D2D37
:1022E0000E944511C7010E9453111F910F91FF9049
:1022F000EF90DF900895A0E0B0E0E1E8F1E10C9408
:10230000112F8CE00E94B00A882379F585E296E0CF
:1023100063E171E00E944E2C5E9A80E00E94960B71
:102320000E94750C5E9821C085E296E00E94CD2D3A
:10233000482F8091AD04882321F0842F0E946C0DDA
:1023400014C080911805E82FF0E031969F012F719D
:10235000307031978091170590E02817390729F0E0
:10236000E251FB4F40832093180585E296E00E94DE
:10237000932D892BC9F680919803843009F08CC085
:102380000E94212960939C0470939D0480939E0475
:1023900090939F04611571058105910561F481E0B9
:1023A00090E0A0E0B0E080939C0490939D04A09303
:1023B0009E04B0939F048091A8049091A904816029
:1023C0009093A9048093A80483E0809398038FE7F7
:1023D0000E948C0AC5EED4E00E94A00A899304E012
:1023E000CE3ED007C9F74091D0048091E504282F54
:1023F00030E0842F90E08227932786FF40C080E45E
:1024000048274093D004C90188739070C89709F594
:1024100010E014C01F5F8091E603E12FF0E084FF1D
:1024200006C0EB51FB4F80810E94980C07C0EB5116
:10243000FB4F85E296E060810E94062E212F30E05E
:102440008091E50490E0877090708217930714F7ED
:1024500016C02F733070232B91F48091E604809383
:10246000A0048091E7048093A2048091E804809303
:10247000A3048091EB048093AA041092AB04809192
:102480001905813019F482E08093190580911905AE
:10249000833011F4109219050E9421295B016C010F
:1024A0008091A4049091A504A091A604B091A704E2
:1024B0000097A105B105C9F0A6019501281B390BAC
:1024C0004A0B5B0BDA01C901885B9B40A040B0401E
:1024D00060F00E94D70A8093A1041092A404109285
:1024E000A5041092A6041092A7048EEB93E00E941C
:1024F0001009209198043091990440919A045091C8
:102500009B0486017501E21AF30A040B150BE6160B
:10251000F7060807190708F4EAC0A0929804B092D9
:102520009904C0929A04D0929B04A8958091AC041F
:10253000883008F0D4C08091AC048F5F8093AC04E5
:10254000E0909C04F0909D0400919E0410919F04E3
:10255000E114F1040105110511F18EEB93E00E94E5
:102560001009AE18BF08C00AD10A6A157B058C0590
:102570009D0588F480919F0384FD04C080ED97E061
:102580000E94060810929C0410929D0410929E04D2
:1025900010929F0404C080E090E00E940608909191
:1025A000D004907C9093D0040091180510911705E9
:1025B0000117B1F180911905823091F590589093EF
:1025C000D0048EEB93E00E940609893010F048E0B9
:1025D00002C0482F415030E013C03F5FA32FB0E04E
:1025E000812F90E0FC01E251FB4F2081FD01E0537F
:1025F000FB4F2083A25FBA4F2C930196182F1F71B7
:10260000341710F4101749F710931705832F895CBE
:102610009091D004892B8093D00430930E051AC07A
:10262000209119052430D1F490910E05EFE0F5E0EA
:10263000A1EDB4E0292F30E02E0F3F1F02C08191A1
:102640008D93E217F307D9F7995C8091D004982B0A
:102650009093D00483E08093190523C08091930464
:10266000823029F491609093D0045E9A0FC09093C9
:10267000D0045E98222319F481E08093190580919B
:102680001905833019F484E080931905F89480913A
:10269000E603877067E273E041ED54E00E9497091A
:1026A00078945D9A809192040E94C10A8EEB93E027
:1026B0000E940609682F80ED94E00E94680FE09167
:1026C0009204EF5FE0939204E83131F0F0E0E254DD
:1026D000FC4F8785882359F41092920408C080919A
:1026E000AC04883009F45E9A89E08093AC04809150
:1026F000E603887171F180919803823051F58091E1
:10270000A8049091A904880F991F9093A90480931D
:10271000A80483E0809398030E94750C0E942129ED
:102720006093A4047093A5048093A6049093A704D7
:10273000611571058105910561F481E090E0A0E0EB
:10274000B0E08093A4049093A504A093A604B09352
:10275000A7048091E60384FF1EC08091A804909195
:10276000A9048E7F0E94340A182F8091A0046091E2
:10277000AA040E94550D082F8091A104612F0E9488
:10278000550D282F8091A2046091A304402F009141
:1027900099030E94E7105D98809193048130C9F0FD
:1027A000813020F0823009F03FC033C08EE00E94BB
:1027B000452A892BC9F581E0809393040E9413294F
:1027C0006093940470939504809396049093970477
:1027D0002BC08EE00E94452A892B21F50E941329E7
:1027E000209194043091950440919604509197045F
:1027F000621B730B840B950B695E734080409040A5
:1028000098F082E08093930480ED97E00E940608A0
:102810000BC08EE00E94452A892B31F080E090E0C9
:102820000E94060810929304CDB7DEB7EAE00C943C
:102830002D2F8CE060E00E94A6298BE061E00E94D1
:10284000A6298DE061E00E94A62982E060E00E9456
:10285000A62984E061E00E94A629089582E0809381
:10286000B00085E08093B10083E061E00E94A6297A
:1028700083E060E00E94122A08951F93182F0E949F
:10288000212960938D0470938E0480938F0490931C
:10289000900410937B04112329F440E855E260E092
:1028A00070E004C040E051EE60E070E085E296E048
:1028B0000E940C2D1F910895ACE1B0E0E2E6F4E136
:1028C0000C94112F0E9421297B018C0181E00E9430
:1028D000960BA4E7AA2E6E010894C11CD11CF3E04C
:1028E000BF2EA982C60161E00E94A40FB092980396
:1028F0000E94750C6AEF70E080E090E00E9447292A
:1029000080919803833009F07DC085E296E00E94B3
:10291000932D892B09F076C00E9421296E197F0919
:10292000800B910B6058734C894C914008F06AC041
:10293000D8CF8FE70E948C0A0E94A00A843509F044
:102940005CC089830E94A00A182F00E010937A04CB
:10295000009379040E94A00A080F111D10937A04B5
:10296000009379040E94A00A809378040E94A00A30
:1029700080937704813108F040C0FF2407C00E9493
:10298000A00A095A1B4FF8018083F3940F2D10E021
:102990008091770490E0880F991F0817190778F342
:1029A00080E78983CE01019661E00E94A40F83E055
:1029B000809398030E94750C62E370E080E090E0E1
:1029C0000E944729809198038330A9F08FE70E94E5
:1029D0008C0A0E94A00A803581F4898303EA13E0FF
:1029E0000E94A00AF80181938F01F3E00E3B1F07BC
:1029F000B9F781E003C082E001C083E06C96EAE0B1
:102A00000C942D2F80919803833009F092CFF3CF4F
:102A100083E00E94B00A8093E70384E00E94B00A3A
:102A20008093E80387E061E00E94B60A6AE070E004
:102A300080E090E00E9447290E94750C00000895F4
:102A40000F931F93082F17C05E9A64E670E080E032
:102A500090E00E9447295E9864E670E080E090E094
:102A60000E9447291F5F101778F36CE271E080E045
:102A700090E00E94472910E0F6CF482F392F25E03B
:102A80000DC0F999FECF1FBA842F932F92BD81BD3F
:102A900060BD0FB6F894FA9AF99A0FBE215059F01A
:102AA000F999FECF842F932F92BD81BDF89A80B5FE
:102AB000681739F7089582E00E9420150895A0E074
:102AC000B0E0E5E6F5E10C940A2F482E562EEE24F0
:102AD000FF2488249924C0E0D0E0CC24DD2436E310
:102AE000332E04C055245394CC24DD24442069F4AF
:102AF00080919903839DE00111242AE9E22E23E0CD
:102B0000F22E99E0892E912C1DC021E0421671F41D
:102B100080919903839DE00111242B968EEBE82E82
:102B200083E0F82E09E2802E912C0CC032E043168F
:102B300049F419E9E12E13E0F12EB1E08B2E912C2E
:102B4000C8EDD0E03E016C0C7D1C10922205109265
:102B50002105E3011BC0552059F4F999FECFD2BDE0
:102B6000C1BDF89A80B5F701E00FF11F808307C05F
:102B7000F701E00FF11FCE0160810E943D150E0D9F
:102B80001F1DF80180810E94560821969E0126197A
:102B9000022F10E008151905F0F2CE015520D9F4E6
:102BA000F999FECFD2BDC1BDF89A20B5F999FECFF3
:102BB0002196D2BDC1BD2197F89A80B590E0B22E82
:102BC000AA248A299B2920912105309122052817C2
:102BD000390759F487CF2196609122050E943D154F
:102BE000CE01609121050E943D1580E091E0C80E64
:102BF000D91E91E0C91693E0D90608F477CF852D48
:102C0000CDB7DEB7E1E10C94262F80E061E00E94B1
:102C10005F1581E061E00E945F15089580E060E04B
:102C20000E945F15882331F081E060E00E945F150B
:102C3000882331F40E94B8080E9473080E94051688
:102C4000089582E061E00E945F15089582E060E0EF
:102C50000E945F1580919903843020F010929903AF
:102C60000E94211608951F93182F0E942616809106
:102C70009903811731F0143020F4109399030E94C6
:102C800021161F9108951092550485E6E0EFF3E0B8
:102C9000DF011D928A95E9F708951F93182F8F374A
:102CA00011F08830E1F5E0915504EE2309F455C0A8
:102CB000E150E0935504F0E0E051FC4F108285E2D2
:102CC00096E06DE00E94062E10E00AC0E12FF0E0D1
:102CD000E051FC4F85E296E060810E94062E1F5F66
:102CE00080915504181790F385E296E060E20E9407
:102CF000062E85E296E06DE00E94062E10E00AC0E6
:102D0000E12FF0E0E051FC4F85E296E060810E9407
:102D1000062E1F5F80915504181790F31CC08B314D
:102D200019F40E9443161FC08D30E9F08A30D9F0A3
:102D300080915504843688F485E296E0612F0E94E4
:102D4000062E80915504E82FF0E0E051FC4F1083EF
:102D50008F5F8093550480E007C085E296E067E0CE
:102D60000E94BA2AF8CF81E01F9108951F93CF9354
:102D7000DF93CDECD3E010E03BC085E296E062E269
:102D800071E00E944B2C85E296E0612F4AE050E012
:102D90000E94C82B85E296E06FE271E00E944B2C06
:102DA000699170E080E090E02091CC0330E040E059
:102DB00050E00E949A2E20E137E240E050E00E946D
:102DC0009A2EDC01CB014091C3035091C403609162
:102DD000C5037091C603480F591F6A1F7B1F85E208
:102DE00096E02AE030E00E948F2B1F5F183119F027
:102DF0008881882311F6DF91CF911F910895EF927A
:102E0000FF920F931F93882339F485E296E066E6DC
:102E10007AE00E94D82A3BC090E00E94CD0824E6C8
:102E200030E040E050E00E94CC2E122F032FF42E11
:102E3000E52E622F732F842F952F2AE030E040E09B
:102E400050E00E94CC2E85E296E0BA01A9012AE06A
:102E500030E00E94802B85E296E06EE20E94BA2A62
:102E6000612F702F8F2D9E2D2AE030E040E050E042
:102E70000E94CC2EAB01BC0185E296E02AE030E056
:102E80000E94802B85E296E063E70E94EC2A1F9166
:102E90000F91FF90EF900895FF920F931F93CF93A0
:102EA000DF9385E296E06CE57AE00E94992A8091B2
:102EB000A303813041F485E296E063E47AE00E9466
:102EC000D82AFF2466C0823029F485E296E06CE2BD
:102ED0007AE0F5CF8430A9F785E296E068E17AE000
:102EE000EECFCF2DD0E0C930D1051CF06F2D685C3E
:102EF00002C06F2D6F5C85E296E00E94BA2A85E2DF
:102F000096E060E17AE00E94992ABE016F5F7F4FF0
:102F100085E296E04AE050E00E94242C85E296E0AB
:102F200065E07AE00E94992A8E010D551C4FD80168
:102F30001196EC91E032F8F485E296E068EF79E0E2
:102F40000E94992AF8018181803130F085E296E073
:102F500063E371E00E944B2CCD55DC4F698170E03A
:102F60006F7070706F5F7F4F85E296E04AE050E0CF
:102F70000E94372C0DC0F0E0EF70F070EE0FFF1FD5
:102F8000E85BFC4F6081718185E296E00E944E2CE7
:102F9000F39480917804F81608F4A3CF85E296E0C4
:102FA0006DED79E00E94992A8091BB030E94FF1683
:102FB00085E296E062EC79E00E94992A8091BC0358
:102FC0000E94FF1685E296E067EA79E00E94992A5E
:102FD0008091BD030E94FF1685E296E06CE879E0DF
:102FE0000E94992A4091B3035091B4036091B503B4
:102FF0007091B603411551056105710539F185E2FE
:1030000096E02AE030E00E948F2B85E296E069E5A9
:1030100079E00E94992A8091B7030E940009AB01D0
:10302000BC0185E296E02AE030E00E948F2B85E229
:1030300096E065E379E00E94992A85E296E0609146
:10304000B8034AE050E00E94DA2B06C085E296E021
:103050006CE279E00E94D82A85E296E06FE079E0A0
:103060000E94992A6091B9037091BA0385E296E0B3
:103070004AE050E00E94B42B85E296E062EF78E0EF
:103080000E94992A6091B203603150F470E06F5F42
:103090007F4F85E296E04AE050E00E94372C06C060
:1030A00085E296E069EE78E00E94D82A85E296E013
:1030B0006CEC78E00E94992A8091B10380FD03C0F6
:1030C00065E371E002C069E371E085E296E00E9489
:1030D0004E2C85E296E06FEA78E00E94992A809172
:1030E000B10382700E94600D85E296E060E978E0AD
:1030F0000E94992A8091B10384700E94600D85E23C
:1031000096E061E778E00E94992A8091B103887087
:103110000E94600DCDB7DEB7E5E00C94322F1F930F
:10312000CF93DF9385E296E060EB7BE00E94992AE3
:103130004091C3035091C4036091C5037091C603CD
:1031400085E296E02AE030E00E948F2B85E296E04F
:103150006AE97BE00E94992A4091C7035091C80315
:103160006091C9037091CA0385E296E020E130E0E6
:103170000E948F2B85E296E064E87BE00E94992A0A
:1031800085E296E06091CB034AE050E00E94DA2BA2
:1031900085E296E06EE67BE00E94992A85E296E061
:1031A0006091CC034AE050E00E94DA2B85E296E081
:1031B00068E57BE00E94992ACDECD3E010E012C0D4
:1031C000112331F085E296E06DE371E00E944B2C13
:1031D00085E296E069914AE050E00E94C82B1F5FAB
:1031E000183119F08881882359F785E296E00E940A
:1031F000C22A85E296E062E47BE00E94992A85E299
:1032000096E06091E5034AE050E00E94DA2B85E207
:1032100096E06DE27BE00E94992AE091E603F0E0FF
:10322000E770F070EE0FFF1FE859FC4F608171816D
:1032300085E296E00E944E2C85E296E068E17BE014
:103240000E94992A8091E60390E0887190708830FE
:10325000910589F0893091051CF4892B39F01BC048
:103260008031910569F04897B1F40FC085E296E08E
:103270006FE07BE00EC085E296E063E07BE009C092
:1032800085E296E06DEF7AE004C085E296E063EFB8
:103290007AE00E94D82A85E296E06FED7AE00E94FB
:1032A000992A4091BF035091C0036091C10370916E
:1032B000C20385E296E02AE030E00E948F2B85E28F
:1032C00096E066EC7AE00E94992A80919F038071D3
:1032D0000E94600D85E296E06DEA7AE00E94992AEC
:1032E00080919F0380740E94600D85E296E064E9FE
:1032F0007AE00E94992A80919F0380720E94600D5B
:1033000085E296E067E77AE00E94992A8EEB93E0E7
:103310000E941009AB01BC0185E296E02AE030E092
:103320000E94802B85E296E062E77AE00E94992A6B
:103330008EEB93E00E9410099B01AC0160E472E403
:103340008FE090E00E94CC2E85E296E0BA01A901C0
:103350002AE030E00E94802B85E296E06FE67AE07A
:103360000E94D82ADF91CF911F910895EF92FF928A
:103370000F931F937C0105E216E0C8016F2D70E0EA
:103380004AE050E00E94A32BC8016EE20E94BA2AD4
:10339000B701E4E076956795EA95E1F76F70707094
:1033A000C8014AE050E00E94A32BC8016EE20E94CF
:1033B000BA2A8FE0E822FF24C801B7014AE050E0B2
:1033C0000E94A32B1F910F91FF90EF9008950F93F0
:1033D0001F93CF93DF932091EF032F3FA9F585E251
:1033E00096E061EF75E00E94992A82E693E00E94E0
:1033F000B61985E296E060ED75E00E94992A809109
:10340000790490917A040E94B61985E296E06DE9FC
:1034100075E00E94D82A85E296E06AE775E00E948E
:10342000D82A85E296E062E675E00E94D82A85E215
:1034300096E06DE375E00E94D82A85E296E00E944E
:10344000C22A0E944C1769C012160CF066C03327BE
:1034500027FD30958091780490E0821793070CF453
:103460005CC085E296E068E275E00E94992A60916E
:10347000EF03772767FD709585E296E04AE050E01C
:103480000E94372C85E296E06DEF74E00E94992A45
:1034900008E210E03AC0C12FD0E0CC0FDD1FC95ABE
:1034A000DB4F288130E08091EF03992787FD9095CD
:1034B00001972817390741F585E296E06FE371E03F
:1034C0000E944B2C85E296E0602F4AE050E00E947B
:1034D000C82B85E296E063E471E00E944B2CE98101
:1034E000F0E0EF70F070EE0FFF1FE85BFC4F6081C3
:1034F000718185E296E00E944B2C85E296E067E4BC
:1035000071E00E944B2C0F5F1F5F809177041817AA
:1035100010F285E296E00E94C22ADF91CF911F91BE
:103520000F910895ACE1B0E0E8E9FAE10C94132FB3
:10353000282F8091EF038F3F09F042C1822F90E046
:10354000FC013A97EF36F10508F033C1EC5CFF4F10
:103550000C94402F85E296E069E471E0AEC085E20C
:1035600096E069E471E00E944E2C1CC185E296E071
:1035700065E571E00E944E2C85E78983DE01129695
:10358000E3EAF3E08BE101900D928150E1F7CE0187
:1035900001966CE10E94A40F0E94750C83E0809359
:1035A000980368EC70E080E090E00E9447298091E9
:1035B0009803843009F0FDC08FE70E948C0A0E94B6
:1035C000A00A8983853509F0F4C085E296E06FEDA5
:1035D00074E00E94D82A85E296E061EC74E00E94D3
:1035E000D82A85E296E063EA74E0ACC085E296E012
:1035F0006DE671E00E944E2C89E68983CE0101962A
:1036000061E00E94A40F0E94750C83E080939803F0
:1036100068EC70E080E090E00E9447298091980378
:10362000843009F0C6C08FE70E948C0A0E94A00A6D
:1036300089838E010E5F1F4F9DE1E92EF12CEC0E68
:10364000FD1E0E94A00AD8018D938D01AE15BF0505
:10365000C1F7A3EAB3E0FE0132968BE101900D922F
:103660008150E1F78981893409F0A3C085E296E0B1
:1036700065E874E00E94D82A85E296E067E674E087
:103680000E94D82A85E296E069E474E05BC085E296
:1036900096E067E871E00E944E2C8EEF8093EF0376
:1036A00088C020522750922F905380917804891718
:1036B00038F485E296E066E971E00E944E2C79C00C
:1036C0009093EF036FC084E18093EF0385E296E06F
:1036D00062E174E037C085E18093EF0385E296E014
:1036E0006BED73E02FC086E18093EF0385E296E0F7
:1036F00064EA73E027C087E18093EF0385E296E0F8
:103700006AE573E01FC088E18093EF0385E296E0ED
:1037100069E473E017C089E18093EF0385E296E0E6
:1037200065E373E00FC08AE18093EF0385E296E0E2
:1037300060E273E007C08BE18093EF0385E296E0DF
:1037400068EF72E00E94D82A34C085E296E06EED00
:1037500072E00E94D82A8091B10391E01DC085E2F9
:1037600096E068EC72E00E94D82A8091B10392E062
:1037700013C085E296E063EB72E00E94D82A809144
:10378000B10394E009C085E296E068E972E00E9426
:10379000D82A8091B10398E089278093B1038FEFF5
:1037A0008093EF030E94E71904C085E296E00E942F
:1037B000CD2D85E296E00E94932D892BB1F763C150
:1037C000822F0E944D16882309F45DC18091550413
:1037D000882321F48FEF8093EF034DC180EF93E0B6
:1037E00060E070E040E050E00E949C069B01AC016C
:1037F0006091EF03862F992787FD9095A92FB92F08
:10380000FC013197EB31F10508F025C1ED55FF4F73
:103810000C94402FE62FFF27E7FDF0958091780468
:1038200090E08E179F070CF416C1DA01C9010197C9
:10383000A109B1098097A105B10540F0FF2410E06E
:1038400008E26F010894C108D10826C0ED55FC4F6D
:10385000822F81508083E7C0612F70E0660F771F51
:10386000695A7B4FFB01808190E08C159D0599F48E
:10387000802F90E0A0E0B0E082179307A407B5077F
:1038800049F4F601ED55FC4FDB0111968C918183D3
:10389000FF24F3940F5F1F5F809177041817E0F205
:1038A000C0C02F3F31054105510511F008F0D3C0CC
:1038B0002093BB03B8C02F3F31054105510511F0DE
:1038C00008F0C9C02093BC03AEC02F3F31054105AD
:1038D000510511F008F0BFC02093BD03A4C0809132
:1038E000F0038062803719F581EF93E060E070E0CB
:1038F00040E050E00E949C069B01AC01DC01CB0142
:103900000197A109B1090897A105B10508F0B6C052
:10391000CA01B90124ED30E340E050E00E949A2E44
:103920009B01AC012A5E3C4A4A46554E24C086366D
:1039300011F581EF93E060E070E040E050E00E941C
:103940009C069B01AC01DC01CB010197A109B109E7
:103950000797A105B10508F091C0CA01B90128EA8D
:1039600031E640E050E00E949A2E9B01AC01245EBB
:103970003C434E46544E211531054105510561F039
:10398000DA01C9018054914EAD49B8418158904F38
:10399000AA4FB24008F05FC02093B3033093B40342
:1039A0004093B5035093B6033EC02F3F3105410508
:1039B000510511F008F04FC02093B70334C0DA016D
:1039C000C9010197A109B1098F3F9105A105B10571
:1039D00008F041C02093B80326C0DA01C901845C15
:1039E0009940A040B0408D549D41A040B04038F473
:1039F0003093BA032093B903FF24F39401C0FF244A
:103A0000211531054105510511F48FEF07C0213112
:103A100031054105510528F4822F81508093B2036E
:103A200002C0FF20C1F0809156048823D1F4809118
:103A3000C7039091C803A091C903B091CA0301962E
:103A4000A11DB11D8093C7039093C803A093C90320
:103A5000B093CA0306C085E296E068EA71E00E946E
:103A60004E2C0E9443168FEF8093EF0385E296E081
:103A70006AE00E94EC2A0E94E71905C021E030E0CC
:103A800040E050E07DCF6C96E8E00C942F2F85E26B
:103A900096E06CE472E00E94D82A85E296E064E346
:103AA00072E00E94D82A85E296E00E94932D892B2D
:103AB00031F085E296E00E94CD2D0E94921A0E947C
:103AC0005C14823019F0833069F405C085E296E019
:103AD00066E172E004C085E296E06FEF71E00E945B
:103AE000D82A08958FEF8093EF03109256040E9416
:103AF000E7190CC085E296E00E94932D892B31F0E6
:103B000085E296E00E94CD2D0E94921A8091EF03EB
:103B10008E3F81F708958091EF03992787FD909557
:103B2000A92FB92FFC013196EB30F10508F074C0D4
:103B3000E254FF4F0C94402F85E296E064E678E073
:103B40000E94D82A82E693E00E94B61985E296E0A8
:103B50006CE478E00E94D82A85E296E067E278E09B
:103B60000E94D82A85E296E06DEF77E00E94D82A7D
:103B700085E296E06CED77E00E94D82A85E296E037
:103B80006FEA77E00E94D82A85E296E069E877E05C
:103B90000E94D82A85E296E065E677E00E94D82A5E
:103BA00085E296E06EE377E00E94D82A85E296E00F
:103BB0000E94C22A0E948F182FC085E296E061E21F
:103BC00077E028C085E296E06CEF76E023C085E2DE
:103BD00096E067EE76E01EC085E296E068EC76E05F
:103BE00019C085E296E064E876E014C085E296E0CC
:103BF0006FE676E00FC085E296E06AE576E00E9427
:103C0000D82A85E296E064E176E004C085E296E099
:103C10006EEF75E00E94D82A6AE070E080E090E0E4
:103C20000E94472904C085E296E00E94CD2D85E2DE
:103C300096E00E94932D892BB1F70895A2E2B0E09F
:103C4000E4E2FEE10C94092F8E010F5F1F4F80E12B
:103C5000D8011D928A95E9F785E296E066EC71E05D
:103C60000E944E2C0E94081520E431EE4DE958E1E7
:103C70002F8F38A349A35AA380EC91EDA8E9BBE1AB
:103C80008B8F9C8FAD8FBE8F24EF31E040E050E0F2
:103C90002F8B388F498F5A8F50E5C52E53ECD52E78
:103CA000E12CF12C40E4442E41EE542E4DE9642EDB
:103CB00048E1742E88249924540133241E8A1D8AD5
:103CC000198A1A8A1B8A1C8AFFC085E296E00E9424
:103CD000CD2D8434B9F0853430F48332B9F18C328F
:103CE00009F0CCC044C0833509F0C8C02F8D38A17D
:103CF00049A15AA1C901DA012C013D018824992466
:103D00005401E2C085E296E064E40E94BA2A85E2AA
:103D100096E040E451EE6DE978E12AE030E00E945F
:103D2000EE2B85E296E06CE20E94BA2A85E296E0EC
:103D300040EC51ED68E97BE12AE030E00E94EE2B97
:103D400085E296E06CE20E94EC2ABEC019821A82DB
:103D50001B821C821D821E821F82188619861A866B
:103D60001B861C861D861E861F86188A3AC03394C1
:103D700034E0331609F0A8C069817A818B819C8177
:103D800028EE33E040E050E00E949A2E6F8F78A337
:103D900089A39AA36D817E818F8198850E949A2E36
:103DA0006B8F7C8F8D8F9E8F89859A85AB85BC8527
:103DB0008F8B988FA98FBA8F6D857E858F85988917
:103DC0000E949A2E6B017C0190E2C9169EE4D906EE
:103DD00090E0E90690E0F90630F48CE162E30E949D
:103DE000B60A332471C0A0E3CA16A5E7DA06A0E03C
:103DF000EA06A0E0FA0618F48CE162E2F0CFB0E443
:103E0000CB16BCE9DB06B0E0EB06B0E0FB0618F42D
:103E10008CE166E2E4CFE0E5CE16E3ECDE06E0E01E
:103E2000EE06E0E0FE0618F48CE162E1D8CFF0E6A1
:103E3000CF16FAEEDF06F0E0EF06F0E0FF0618F42A
:103E40008CE165E1CCCF20E7C21621E1D20621E06A
:103E5000E20620E0F20618F48CE161E0C0CF30EA1F
:103E6000C31636E8D30631E0E30630E0F30618F473
:103E70008CE163E0B4CF8CE165E0B1CF30ED232E6F
:103E8000280E49E0421500F1032D10E0000F111F2C
:103E9000000F111F81E090E08C0F9D1F080F191F6C
:103EA000D8016D917D918D919C912AE030E040E0A8
:103EB00050E00E949A2E620D711D811D911DF80126
:103EC000608371838283938385E296E00E94932DC1
:103ED000892B09F0FACE81149104A104B10489F46C
:103EE000C301B2010E942C0B61E070E080E090E021
:103EF0000E944729FFEFFE8B1D8A198A1A8A1B8AA6
:103F00001C8A2F89388D498D5A8D82169306A406F6
:103F1000B506E0F40E94D70A29893A894B895C8961
:103F2000280F311D411D511D298B3A8B4B8B5C8B0A
:103F30003D89381708F48D8B4E89841708F48E8BD1
:103F40000894811C911CA11CB11C56C0C301B20174
:103F500028EE33E040E050E00E94CC2E85E296E06F
:103F6000BA01A9012AE030E00E94802B85E296E0A8
:103F70006CE20E94BA2A85E296E06D894AE050E040
:103F80000E94C82B85E296E06CE20E94BA2A6989F9
:103F90007A898B899C89A50194010E94CC2E85E2A7
:103FA00096E0BA01A9012AE030E00E94802B85E268
:103FB00096E06CE20E94BA2A85E296E06E894AE0B9
:103FC00050E00E94C82B85E296E06CE20E94EC2A49
:103FD0004C0C5D1C6E1C7F1C8B8D9C8DAD8DBE8D25
:103FE00084159505A605B70520F44F8C58A069A047
:103FF0007AA08824992454012F8D38A149A15AA16F
:10400000285E33404040504009F05ECFA296E2E186
:104010000C94252FAAE5B0E0E0E1F0E20C94152F16
:104020008B017A018B3009F425C18C3040F5853045
:1040300009F484C0863080F4823009F459C083309A
:1040400020F4813009F044C242C0833009F461C0D9
:10405000843009F03DC265C0883009F49DC08930C4
:1040600038F4863009F486C0873009F031C28CC03C
:10407000893009F499C08A3009F02AC2C9C089364A
:1040800009F476C18A3680F4863609F421C1873670
:1040900020F4853609F01CC202C1873609F431C10B
:1040A000883609F015C235C18C3609F4B8C18D3691
:1040B00038F48A3609F467C18B3609F009C2A3C106
:1040C0008D3609F4E0C1873C09F002C2F4C181E0F9
:1040D00069E270E00E945C110EEB13E0F80181913F
:1040E0008F010E944511F3E0073E1F07B9F7F8C1A1
:1040F00082E06BE170E00E945C1103EA13E0F801DA
:1041000081918F010E944511F3E00E3B1F07B9F723
:10411000E7C183E061E070E00E945C110E945C14E2
:10412000DDC184E061E070E00E945C1181E00E94EA
:1041300045110E943E110E941E1ED4C16091770459
:1041400070E0660F771F85E00E945C1100E010E0D0
:1041500008C0F801E95AFB4F80810E9445110F5FAA
:104160001F4F8091770490E0880F991F0817190757
:1041700080F3B6C186E062E070E00E945C1182E6E6
:1041800093E00E945311ACC187E061E070E00E94AF
:104190005C1180917804A2C188E061E070E00E9427
:1041A0005C11809199039AC186E68983CE010196BC
:1041B00061E00E94A40F0E94750C83E08093980335
:1041C00068EC70E080E090E00E94472980919803BD
:1041D0008430E1F48FE70E948C0A0E94A00A898350
:1041E000863471F489E060E270E00E945C1110E0B6
:1041F0000E94A00A0E9445111F5F1032C9F770C1CA
:1042000089E061E070E00E945C11BBC089E061C19F
:104210008AE069E070E00E945C1110929A0380913C
:104220008F05882351F080919F039091A003A09166
:10423000A103B091A203806809C080919F0390916F
:10424000A003A091A103B091A2038F7780939F0355
:104250009093A003A093A103B093A2030AE913E0F3
:10426000F80181918F010E944511F3E0033A1F0785
:10427000B9F736C18BE060E270E00E945C11F894FF
:1042800000E010E0F801E95DFC4F80810E944511DB
:104290000F5F1F4F00321105A9F7789421C185E601
:1042A00061E070E00E945C110932110509F015C14E
:1042B00020E030E0F901E254FC4FD701A20FB31F18
:1042C0008C9180832F5F3F4F2932310599F759C078
:1042D00086E661E070E00E945C110B31110509F087
:1042E000FCC020E030E0F901ED55FC4FD701A20FF2
:1042F000B31F8C9180832F5F3F4F2B31310599F78E
:1043000040C087E661E070E00E945C110E940516E3
:1043100038C088E661E070E00E945C1185E78A831E
:10432000DE011396E3EAF3E08BE101900D928150F8
:10433000E1F7CE0102966CE10E94A40F0E94750C79
:1043400083E08093980360E273E080E090E00E9455
:10435000472980919803843009F0BFC08FE70E94FD
:104360008C0A0E94A00A8A83853509F0B6C009C06C
:1043700089E661E070E00E945C110E9473080E946F
:10438000B80881E0ABC08AE661E070E00E945C1191
:1043900089E68E8FCE014E9661E00E94A40F0E94A6
:1043A000750C83E08093980360E273E080E090E016
:1043B0000E94472980919803843009F08EC08FE7CE
:1043C0000E948C0A0E94A00A8E8F8E01015E1F4FF0
:1043D0006AE3E62EF12CEC0EFD1E0E94A00AF80105
:1043E00081938F01EE15FF05C1F7A3EAB3E0FE014B
:1043F0007F968BE101900D928150E1F78E8D89348B
:1044000009F06BC0BECF8BE661E070E00E945C11EA
:10441000F70180810E9433160E940E16B2CF8CE6FF
:1044200061E070E00E945C110032110571F487E6D2
:104430008AAFDE01DB96F70180E201900D92815098
:10444000E1F7CE01CA9661E205C087E48AAFCE01EA
:10445000CA9661E00E94A40F0E94750C83E08093CD
:1044600098036CE474E080E090E00E94472980911A
:104470009803843091F58FE70E948C0A0E94A00A6D
:10448000873459F57ECF8DE661E070E00E945C11C3
:104490000930110511F520E030E0F901E656FC4F36
:1044A000D701A20FB31F8C9180832F5F3F4F29301C
:1044B000310599F766CF87EC61E070E00E945C11EE
:1044C00081E00E9445110E943E111092ED030AC046
:1044D0008AEC61E070E00E945C1180E00E9445116E
:1044E0000E943E11C65ADF4FE6E00C94312FA0E047
:1044F000B0E0EDE7F2E20C94112F84E0A82E06E084
:10450000B02E15E0C12E03E215E0B4E6DB2EA2E0EA
:10451000EA2EF3E0FF2EA1C085E296E00E94CD2DA9
:10452000982F80938E0580918D05833021F1843002
:1045300028F4813099F08230B8F409C0853009F44C
:1045400048C0853020F1863009F087C05FC0953BB8
:1045500009F083C081E080938D057FC0923609F019
:104560007AC0E0928D0579C090938C0590938B056D
:10457000F0928D0572C09093890510928A05809102
:104580008B05892780938B05A0928D0566C0D92F56
:10459000C0E02091890530918A052C2B3D2B30936A
:1045A0008A052093890580918B05892780938B0547
:1045B000C0928D052536310508F44FC08CEC61E0C2
:1045C00070E00E945C1181E00E9445110E943E1142
:1045D00042C02091870530918805F901ED5DFA4FC1
:1045E000908380918B05892780938B052F5F3F4FA8
:1045F00030938805209387058091890590918A05DD
:104600002817390750F1B0928D0527C080918B058E
:10461000891759F4609187057091880580918C0500
:1046200043E255E00E940A200DC08BEC62E070E08E
:104630000E945C1180918C050E9445118091EE03CF
:104640000E944511F8018D2D11928A95E9F710927B
:1046500088051092870510928D0585E296E00E94EC
:10466000932D892B09F058CFCDB7DEB7EAE00C9433
:104670002D2F81E08093ED0308C085E296E00E9433
:10468000932D892B11F00E9477228091ED038823CE
:10469000A1F70895A0E0B0E0E0E5F3E20C94142F58
:1046A0000E9421296115710581059105C9F30E94B8
:1046B00093061092C7031092C8031092C903109278
:1046C000CA03DD24E090C703F090C8030091C9033A
:1046D0001091CA03102F0F2DFE2CEE240E948E067F
:1046E0002FEF30E040E050E00E94EE2EE60EF71E85
:1046F000081F191FE092C703F092C8030093C90373
:104700001093CA03D39444E0D416E1F6CDECD3E081
:1047100000E010E090E1E92E97E2F92E4EC00F5F25
:1047200019F40E9473084DC00E948E0622E330E007
:1047300040E050E00E94EE2E6F5FEDECF3E090E081
:1047400004C08191861759F39F5F9117D0F3809130
:10475000CC0390E08E9D90018F9D300D9E9D300D7D
:104760001124862F90E0AC01249FC001259F900D5D
:10477000349F900D1124AA2797FDA095BA2F209160
:10478000C3033091C4034091C5035091C603820F07
:10479000931FA41FB51F20919B0330919C03409150
:1047A0009D0350919E03281739074A075B0708F4B9
:1047B000B6CF69931F5F183121F08881882309F0F3
:1047C000AECFCDB7DEB7E7E00C94302F1F9310913A
:1047D000EF031F3F09F0F1C0893409F467C08A3440
:1047E00028F5883309F479C0893368F4803309F4F3
:1047F00086C0813308F06FC08B3109F44DC081321F
:1048000009F0D5C03DC0813409F49AC0823438F42F
:10481000893309F472C0803409F0C9C031C08234D0
:1048200009F4A1C0863409F0C2C052C0823609F42E
:104830009AC0833690F4883579F1893538F4823519
:1048400009F43FC0833509F0B2C01FC08A3509F4AE
:10485000A9C0813609F0ABC073C0823791F18337AC
:1048600030F48636A9F1893609F0A1C01FC0883717
:1048700099F08A3709F496C0833709F098C005C0CB
:1048800085E296E069E471E019C00E94051685E2B0
:1048900096E063ED71E006C00E940E1685E296E098
:1048A0006DEE71E00E944E2C8EEF7FC00E94730867
:1048B0000E94B80885E296E06CE072E00E944E2CFF
:1048C00076C00E944A2385E296E065E272E0F6CF68
:1048D0000E94B6166CC0805368C085E296E06CEE0C
:1048E00071E00E94D82A9091E603892F885F887131
:1048F000977E892B8093E60320C089E056C085E22D
:1049000096E069ED71E00E94D82A80919F03909112
:10491000A003A091A103B091A20320E130E040E008
:1049200050E082279327A427B52780939F03909375
:10493000A003A093A103B093A2031093EF0337C089
:1049400085E296E063EC71E00E94D82A80919F0393
:104950009091A003A091A103B091A20320E430E0C4
:1049600040E050E012C085E296E062EB71E00E9408
:10497000D82A80919F039091A003A091A103B091A8
:10498000A20320E230E040E050E082279327A427F2
:10499000B52780939F039093A003A093A103B093A6
:1049A000A20302C00E94471D8FEF8093EF03809106
:1049B000EF038E3F09F4DDC0D4C00E944D1688235A
:1049C00009F4D7C080915504882321F48FEF809398
:1049D000EF03C7C080EF93E060E070E040E050E09C
:1049E0000E949C069B01AC018091EF03992787FDF3
:1049F0009095A92FB92FFC013197E930F10508F006
:104A00008CC0E753FF4F0C94402FDA01C901815449
:104A1000914EAD49B8418F57904FAA4FB24008F020
:104A20007CC02093C3033093C4034093C5035093C9
:104A3000C6039AC02093C7033093C8034093C903A9
:104A40005093CA0381E0809356048EC0283031050C
:104A50004105510508F061C02093CB0385C0DA0100
:104A6000C9010197A109B1090A97A105B10508F08B
:104A700054C02093CC0378C080EF93E06DE371E0E5
:104A80000E94B80710E00EC0183130F4E12FF0E0BA
:104A9000E254FC4F87871F5F80E090E06DE371E098
:104AA0000E94B807009759F00E949A07009761F793
:104AB00006C0E12FF0E0E254FC4F17861F5F18316B
:104AC000C0F352C0253031054105510530F5209322
:104AD000E5034AC0DA01C9010197A109B1090697A6
:104AE000A105B105D0F48091E603887F822B8093E5
:104AF000E6033AC0DA01C9010197A109B109805062
:104B0000924CA140B04048F42093BF033093C003BF
:104B10004093C1035093C20327C085E296E068EA40
:104B200071E00E944E2C13C08091C7039091C8037E
:104B3000A091C903B091CA030196A11DB11D809334
:104B4000C7039093C803A093C903B093CA030E94FC
:104B500043168FEF8093EF0385E296E06AE00E94B0
:104B6000EC2A0E948B1D05C0809156048823E1F237
:104B7000EECF1F9108958FEF8093EF0310925604AC
:104B80000E948B1D0CC085E296E00E94932D892B1C
:104B900031F085E296E00E94CD2D0E94E6238091BF
:104BA000EF038E3F81F76AE070E080E090E00E94C2
:104BB000472904C085E296E00E94CD2D85E296E06B
:104BC0000E94932D892BB1F70895AAE2B0E0EBEE95
:104BD000F5E20C940E2F0E9413297B018C0181E0D9
:104BE0000E94960B04C085E296E00E94CD2D85E2DE
:104BF00096E00E94932D892BB1F75E98DD24D39423
:104C000052E6752E42E0842E912C8C0E9D1E5E0184
:104C10000894A11CB11C33E0C32E0E94132920E08C
:104C200030E06E197F09800B910B693C710581059D
:104C3000910510F021E030E08D2D90E028233923FC
:104C4000232B99F10E9413297B018C015D9A80ED41
:104C500097E00E9406087982D401EEEBF3E089E246
:104C600001900D928150E1F7C5016AE20E94A40F04
:104C70005D9880E090E00E940608C09298030E9430
:104C8000750C62E370E080E090E00E94472980911B
:104C90009803843051F4C09298038FE70E948C0AE5
:104CA0000E94A00A823409F4DD248EE00E94452A85
:104CB000892B49F5DD24D39426C05E9A5D9A85E25E
:104CC00096E00E94CD2D8D30910569F08E309105D2
:104CD0001CF40A97B1F407C08332910569F082345D
:104CE000910579F40CC085E296E064EA71E00E94D7
:104CF000D82A0E94BB2505C00E941E1E02C00E9429
:104D000039235E985D9885E296E00E94932D892B69
:104D100009F483CFD2CF8F929F92AF92BF92CF925E
:104D2000DF92EF92FF920F931F938EE00E94452A2D
:104D3000892B09F083C068EC70E080E090E00E946D
:104D4000472980E090E00E9406080E9413295B0139
:104D50006C0160ECE62E62E1F62E012D112DEA0CBD
:104D6000FB1C0C1D1D1D06C08EE00E94452A892BD0
:104D700009F062C00E9413296E157F058007910714
:104D800098F38EE00E94452A892B09F055C080EDEA
:104D900097E00E9406080E9413297B018C01992448
:104DA0009394882488E496E2A0E0B0E0A80EB91EAF
:104DB000CA1EDB1E29C0AE14BF04C006D10638F4DB
:104DC00080ED97E00E940608882483941DC00E940D
:104DD00013296E197F09800B910B693C71058105C0
:104DE000910590F00E9413297B018C0180E09920AD
:104DF00009F481E0982E882319F480E090E002C045
:104E000080ED97E00E9406088EE00E94452A892BDB
:104E100091F280E090E00E940608882049F080919D
:104E200099038F5F83700E9433160E940E1606C08E
:104E30000E944A230E9405160E94E5251F910F91AA
:104E4000FF90EF90DF90CF90BF90AF909F908F90AA
:104E5000089580E067EF77E042E050E00E944E283E
:104E60000895EF92FF920F931F9380E00E943F08F6
:104E70000E94191489E061E00E94A62989E060E09F
:104E80000E94122A86E061E00E94A62985E061E086
:104E90000E94A6298EE060E00E94A62988E060E0DA
:104EA0000E94A62988E061E00E94122A81E161E067
:104EB0000E94A62981E160E00E94122A0E942E141D
:104EC00085E296E040E052EC61E070E00E940C2D3B
:104ED0000E9426160E940E160E943A0D8FEF8093B4
:104EE000AC040E94292778940E9413297B018C012D
:104EF0008091AC048F3F09F0C7C00E9413296E193E
:104F00007F09800B910B605D77408040904008F0F6
:104F1000BBC0EECF85E296E00E94CD2D85E296E003
:104F20000E94932D892BB1F785E296E062E472E04E
:104F30000E944B2C82E693E00E94B61985E296E02F
:104F400069E572E00E944B2C85E296E064E070E037
:104F50004AE050E00E94372C62E370E080E090E08D
:104F60000E94472985E296E00E94932D04970CF158
:104F700085E296E00E94CD2D82349105D1F485E240
:104F800096E00E94CD2D8E34910599F485E296E04D
:104F90000E94CD2D8434910561F485E296E00E9453
:104FA000CD2D819731F480E090E00E9406080E94A8
:104FB000E5254091BF035091C0036091C1037091FA
:104FC000C203DB01CA010197A109B1090497A10538
:104FD000B10568F44093AD04433029F040E052EC51
:104FE00061E070E004C040EA56E861E070E085E20C
:104FF00096E00E940C2D0E948B265E9880E090E047
:105000000E9406080E943A0D80E00E94960B809153
:1050100092040E94C10A0E94750C1092170510920A
:1050200018051092190510E015C062E370E080E0E9
:1050300090E00E94472980ED97E00E94060862E315
:1050400070E080E090E00E94472980E090E00E94BC
:1050500006081F5F80919903811738F78091E60356
:1050600090E084FF09C020E088719070489709F4AF
:1050700021E0822F0E943D148FE00E943F081F9183
:105080000F91FF90EF90089580ED97E00E94060841
:105090008EE061E00E94122A5E9A40CF823000F5D5
:1050A000E82FF0E0EE0FFF1FE057FA4F71836083A7
:1050B000882319F08130A1F408C0809169008C7FA9
:1050C000842B80936900E89A089580916900440FC9
:1050D000551F440F551F837F842B80936900E99AE5
:1050E00008951F920F920FB60F9211242F933F93A2
:1050F0004F935F936F937F938F939F93AF93BF93E0
:10510000EF93FF938091900590919105892B29F061
:10511000E0919005F09191050995FF91EF91BF9174
:10512000AF919F918F917F916F915F914F913F913F
:105130002F910F900FBE0F901F9018951F920F92F6
:105140000FB60F9211242F933F934F935F936F935A
:105150007F938F939F93AF93BF93EF93FF93809130
:10516000920590919305892B29F0E0919205F09199
:1051700093050995FF91EF91BF91AF919F918F9109
:105180007F916F915F914F913F912F910F900FBE43
:105190000F901F9018951F920F920FB60F92112427
:1051A0002F933F938F939F93AF93BF9380919805D5
:1051B00090919905A0919A05B0919B0530919C051D
:1051C0000196A11DB11D232F2D5F2D3720F02D57E6
:1051D0000196A11DB11D20939C0580939805909385
:1051E0009905A0939A05B0939B05809194059091A1
:1051F0009505A0919605B09197050196A11DB11D49
:105200008093940590939505A0939605B093970588
:10521000BF91AF919F918F913F912F910F900FBEB2
:105220000F901F9018958FB7F894209198053091A2
:10523000990540919A0550919B058FBFB901CA010C
:1052400008959FB7F8942091940530919505409169
:1052500096055091970586B5A89B06C08F3F21F013
:105260002F5F3F4F4F4F5F4F9FBF542F432F322F22
:105270002227280F311D411D511D82E0220F331FAF
:10528000441F551F8A95D1F7B901CA010895EF92BD
:10529000FF920F931F93CF93DF937B018C010E94AA
:1052A0002129EB010EC00E9421296C1B7D0B685E39
:1052B0007340C8F30894E108F10801091109C851C5
:1052C000DC4FE114F1040105110569F7CDB7DEB734
:1052D000E6E00C94312F789484B5826084BD84B567
:1052E000816084BD85B5826085BD85B5816085BDE1
:1052F000EEE6F0E0808181608083E1E8F0E01082FA
:10530000808182608083808181608083E0E8F0E03A
:10531000808181608083E1EBF0E080818460808324
:10532000E0EBF0E0808181608083EAE7F0E080815B
:1053300084608083808182608083808181608083BB
:105340008081806880831092C1000895CF93DF939D
:10535000482F50E0CA018850944FFC0134914C51C1
:10536000544FFA018491882369F190E0880F991FC6
:10537000FC01EA53F44FA591B491FC01E053F44FC2
:10538000C591D491662351F42FB7F8948C91932F43
:10539000909589238C93888189230BC0623061F4B6
:1053A0002FB7F8948C91932F909589238C938881B3
:1053B000832B88832FBF06C09FB7F8948C91832BD3
:1053C0008C939FBFDF91CF910895833071F084302B
:1053D00028F48130A1F0823021F514C08630B1F07C
:1053E0008730D1F08430E9F404C0809180008F7759
:1053F00003C0809180008F7D80938000089584B5E4
:105400008F7702C084B58F7D84BD08958091B000F0
:105410008F778093B00008958091B0008F7D809346
:10542000B0000895FF920F931F93F62E482F50E07F
:10543000CA01845F934FFC012491CA018850944FA4
:10544000FC0114914C51544FFA0104910023C9F00E
:10545000222319F0822F0E94E529E02FF0E0EE0FC1
:10546000FF1FE053F44FA591B4919FB7F894FF202C
:1054700021F48C911095812302C08C91812B8C9307
:105480009FBF1F910F91FF9008950F931F93482F77
:1054900050E0CA01845F934FFC012491CA018850F7
:1054A000944FFC0104914C51544FFA011491112373
:1054B00019F420E030E015C0222319F0822F0E9459
:1054C000E529812F90E0880F991F8652944FFC01A7
:1054D000A591B4918C9120E030E0802311F021E07F
:1054E00030E0C9011F910F910895A0E0B0E0EBE713
:1054F000FAE20C94132F7C016B018A01C0E0D0E02A
:105500000FC0D6016D916D01D701ED91FC91019015
:10551000F081E02DC7010995C80FD91F0150104037
:105520000115110571F7CE01CDB7DEB7E8E00C9497
:105530002F2FEF92FF920F931F93CF93DF937C0156
:105540008B01C0E0D0E0F8010F5F1F4F649166232C
:1055500059F0D701ED91FC910190F081E02DC70148
:105560000995C80FD91FEFCFCE01CDB7DEB7E6E062
:105570000C94312FDC01ED91FC910190F081E02D34
:1055800009950895EF92FF920F931F938C016DE0A0
:105590000E94BA2A7C01C8016AE00E94BA2A9C01D2
:1055A0002E0D3F1DC9011F910F91FF90EF9008959F
:1055B000EF92FF920F931F937C010E94992A8C0116
:1055C000C7010E94C22A9C01200F311FC9011F91EF
:1055D0000F91FF90EF900895EF92FF920F931F931A
:1055E0007C010E94BA2A8C01C7010E94C22A9C0138
:1055F000200F311FC9011F910F91FF90EF90089567
:10560000CF93DF93EC016115710519F420E030E0D0
:105610000FC0DB010D900020E9F71197A61BB70B17
:10562000E881F9810280F381E02DAD0109959C01AB
:10563000C901DF91CF9108954F925F927F928F922F
:105640009F92AF92BF92CF92DF92EF92FF920F9311
:105650001F93DF93CF93CDB7DEB7A1970FB6F89422
:10566000DEBF0FBECDBF2C01742ECB01223008F45B
:105670002AE019A231E2C32ED12CCC0EDD1E822EDF
:105680009924AA24BB24672D752FA50194010E949B
:10569000CC2E79018A01C801B701A50194010E94AD
:1056A0009A2E472D461B0894C108D1084A3010F4A1
:1056B000405D01C0495CF6014083E114F10401053D
:1056C000110521F07E2C5F2DC801DDCFC201B6018E
:1056D0000E94002BA1960FB6F894DEBF0FBECDBF7F
:1056E000CF91DF911F910F91FF90EF90DF90CF90BE
:1056F000BF90AF909F908F907F905F904F90089554
:10570000DC012115310541F4ED91FC910190F0810E
:10571000E02D642F099508950E941C2B0895EF92A7
:10572000FF920F931F937C010E94802B8C01C70175
:105730000E94C22A9C01200F311FC9011F910F91A5
:10574000FF90EF900895EF92FF920F931F939A01AD
:105750007B0100E010E0B801A7010E94802B1F919F
:105760000F91FF90EF900895EF92FF920F931F9388
:105770007C010E94A32B8C01C7010E94C22A9C01BC
:10578000200F311FC9011F910F91FF90EF900895D5
:10579000EF92FF920F931F939A01E62EFF2400E0F1
:1057A00010E0B801A7010E94802B1F910F91FF907C
:1057B000EF900895EF92FF920F931F937C010E9448
:1057C000C82B8C01C7010E94C22A9C01200F311FE7
:1057D000C9011F910F91FF90EF900895A0E0B0E0F4
:1057E000E4EFFBE20C94132FEC016A017B0121151D
:1057F000310541F4E881F9810190F081E02D642FB9
:1058000009951BC02A303105B1F477FF13C06DE252
:105810000E94BA2A8C0144275527BA014C195D0908
:105820006E097F09CE012AE00E941C2B9C01200FEB
:10583000311F04C02AE00E941C2B9C01C901CDB776
:10584000DEB7E8E00C942F2FEF92FF920F931F9397
:105850007B019A010027F7FC0095102FB801A701E2
:105860000E94EE2B1F910F91FF90EF900895EF9201
:10587000FF920F931F937C010E94242C8C01C7017F
:105880000E94C22A9C01200F311FC9011F910F9154
:10589000FF90EF9008950E94002B0895EF92FF92E1
:1058A0000F931F937C010E944B2C8C01C7010E9417
:1058B000C22A9C01200F311FC9011F910F91FF9037
:1058C000EF90089508951F920F920FB60F92112432
:1058D0002F933F934F938F939F93EF93FF938091D9
:1058E000C00082FD1DC04091C6002091DD053091B1
:1058F000DE052F5F3F4F2F7330708091DF05909151
:10590000E0052817390771F0E091DD05F091DE051B
:10591000E356FA4F40833093DE052093DD0502C045
:105920008091C600FF91EF919F918F914F913F9190
:105930002F910F900FBE0F901F9018951F920F92EE
:105940000FB60F9211242F933F938F939F93EF9352
:10595000FF93209121063091220680912306909199
:1059600024062817390731F48091C1008F7D809378
:10597000C10014C0E0912306F0912406EF51FA4FC4
:105980002081809123069091240601968F73907058
:1059900090932406809323062093C600FF91EF91F5
:1059A0009F918F913F912F910F900FBE0F901F905D
:1059B0001895A0E0B0E0EFEDFCE20C940F2FFC0195
:1059C0001382128288EE93E0A0E0B0E08483958396
:1059D000A683B7838AE893E0918380837587648781
:1059E00057874687318B208B138B028BF58AE48A8D
:1059F000D78AC68AB18EA08E938E828E8F85848F31
:105A00008889858F8989868F8A89878F8B8980A3EA
:105A10002096ECE00C942B2FAF92BF92DF92EF9286
:105A2000FF920F931F93CF93DF93EC017A018B01C9
:105A3000DD24403081EE580780E0680780E0780779
:105A400011F0DD24D39491E0A92EB12CEC89FD89CD
:105A5000DD2069F0C50108A002C0880F991F0A94D3
:105A6000E2F7808360E079E08DE390E005C010828A
:105A700060E874E88EE190E0A80197010E94CC2EC6
:105A800021503040404050405695479537952795D6
:105A900080E12030380720F0DD2011F0DD24D6CF62
:105AA000E889F9893083EA89FB89208319A2EE8984
:105AB000FF89408121E030E0C9010C8C02C0880FD1
:105AC000991F0A94E2F7482B4083EE89FF894081B1
:105AD000C9010D8C02C0880F991F0A94E2F7482B68
:105AE0004083EE89FF894081C9010E8C02C0880F76
:105AF000991F0A94E2F7482B4083EE89FF89808141
:105B00000F8C02C0220F331F0A94E2F7209528233E
:105B10002083DF91CF911F910F91FF90EF90DF9045
:105B2000BF90AF900895DC011C96ED91FC911D97FC
:105B3000E05CFF4F2191319180819181281B390BCD
:105B40002F733070C901089585E296E00E94932D6D
:105B5000892B11F00E94622C0895DC011C96ED91B6
:105B6000FC911D97E05CFF4F20813181E054F040B3
:105B7000DF01AE5BBF4F8D919C91119728173907BC
:105B800019F42FEF3FEF07C08D919C91E80FF91F9B
:105B90008081282F30E0C9010895DC011C96ED9129
:105BA000FC911D97E05CFF4F20813181E054F04073
:105BB000DF01AE5BBF4F8D919C911197281739077C
:105BC00019F42FEF3FEF10C08D919C911197E80FC2
:105BD000F91F20818D919C91119701968F73907080
:105BE00011969C938E9330E0C9010895DC01919643
:105BF0008C919197882339F05496ED91FC915597AB
:105C0000808186FFF9CF91961C920895CF93DF9300
:105C1000EC01EE85FF85E05CFF4F20813181E0548F
:105C2000F0402F5F3F4F2F733070DF01AE5BBF4FEF
:105C30008D919C91119728173907D1F3E05CFF4FA4
:105C400080819181E054F040E80FF91F6083EE8578
:105C5000FF85E05CFF4F31832083EE89FF8920813F
:105C600081E090E00F8C02C0880F991F0A94E2F740
:105C7000282B208381E089A3EC89FD8980818064C1
:105C8000808381E090E0DF91CF9108958F929F9281
:105C9000AF92BF92CF92DF92EF92FF920F931F933A
:105CA00000D000D00F92EDB7FEB7319684E0ADB7CB
:105CB000BEB711968C9383E0818387E0828385E071
:105CC000838381E0848385E296E06DE975E041EEAF
:105CD00055E025EC30E004EC10E0B0ECEB2EF12CBC
:105CE000A1ECCA2ED12CF2ECAF2EB12CE6EC8E2E0C
:105CF000912C0E94D92C0F900F900F900F900F9025
:105D00001F910F91FF90EF90DF90CF90BF90AF90D9
:105D10009F908F900895CF93DF930E946B290E94EC
:105D20003127C4EADDE20E947B112097E1F30E9453
:105D3000A42DF9CF629FD001739FF001829FE00DE7
:105D4000F11D649FE00DF11D929FF00D839FF00DFA
:105D5000749FF00D659FF00D9927729FB00DE11DA6
:105D6000F91F639FB00DE11DF91FBD01CF01112483
:105D7000089597FB092E07260AD077FD04D086D018
:105D800006D000201AF4709561957F4F0895F6F7BC
:105D9000909581959F4F0895A1E21A2EAA1BBB1BD7
:105DA000FD010DC0AA1FBB1FEE1FFF1FA217B307E7
:105DB000E407F50720F0A21BB30BE40BF50B661FFD
:105DC000771F881F991F1A9469F7609570958095C1
:105DD00090959B01AC01BD01CF01089597FB092E61
:105DE00005260ED057FD04D0D7DF0AD0001C38F4AA
:105DF00050954095309521953F4F4F4F5F4F0895F7
:105E0000F6F790958095709561957F4F8F4F9F4FD6
:105E100008952F923F924F925F926F927F928F924E
:105E20009F92AF92BF92CF92DF92EF92FF920F9329
:105E30001F93CF93DF93CDB7DEB7CA1BDB0B0FB633
:105E4000F894DEBF0FBECDBF09942A8839884888F0
:105E50005F846E847D848C849B84AA84B984C88486
:105E6000DF80EE80FD800C811B81AA81B981CE0F7D
:105E7000D11D0FB6F894DEBF0FBECDBFED01089562
:105E8000EE0FFF1F0590F491E02D0994AA1BBB1B98
:105E900051E107C0AA1FBB1FA617B70710F0A61B2A
:105EA000B70B881F991F5A95A9F780959095BC014B
:105EB000CD010895911106C0803219F089508550A6
:0E5EC000D0F70895992788270895F894FFCF0A
:105ECE004E6F005965730054582074696D656F7577
:105EDE007421006D6F64756C65206C6F636B656407
:105EEE003F00486F70206368616E6E656C20002005
:105EFE0040200053004E2F4100386368002C002CC8
:105F0E00205B005D20280029004E4F5420454E4155
:105F1E00424C45440053656E64696E672073657428
:105F2E0074696E677320746F2052580A005265733D
:105F3E00657474696E672073657474696E67732017
:105F4E006F6E2052580A0041626F7274656420654C
:105F5E00646974730A00696E76616C696420736596
:105F6E006C656374696F6E000D0A496E76616C69BB
:105F7E006420696E707574202D206469736361727C
:105F8E006465642107007363616E6E6572206D6FC8
:105F9E0064650053657474696E677320736176650A
:105FAE006420746F20454550524F4D0A005265765D
:105FBE0065727465642073657474696E67732066A8
:105FCE00726F6D20454550524F4D0A004C6F616403
:105FDE00656420666163746F7279206465666175AD
:105FEE006C74730A004B657920616E64206368617E
:105FFE006E6E656C732072616E646F6D697A656426
:10600E000A004F70656E4C52536E672054582073C1
:10601E0074617274696E672000206F6E204857207D
:10602E000050504D005253534900534441005343C6
:10603E004C00525844005458440041494E004C42C2
:10604E004545500053504B54524D0053425553004A
:10605E0053554D44004C4C494E440000342B3400F3
:10606E003800382B340031320031322B34003136C7
:10607E000001000000C01200001A400AA1204EA527
:10608E00001B1E27522C23308025000005400AA13C
:10609E00204EA50020244EA52C2330004B000006D8
:1060AE00400AD0009D49007B289D492C233000E1F9
:1060BE00000005400A4501D7DC03B81E0EBF0023C1
:1060CE002E48E801008A400A6001555502AD1E2097
:1060DE00000023C88025000005400AA1204EA5001F
:1060EE0020244EA52C2330000200020002000200E4
:1060FE000200020002000200020002000200020082
:10610E0002000200020002FF610265026A026E02D4
:10611E00720276027A027E0284028B02900295024D
:10612E009B029B029B029B0235019C02A002A202D3
:10613E00A602A902AE02350100070B0C10111500C4
:10614E00160A1322312900000000062E752A932DFF
:06615E00CD2DAD2DF62D44
:00000001FF
